:020000040800F2
:1000000000800020E50C00082F0D00086B0D000893
:1000100000000000000000000000000000000000E0
:10002000000000000000000000000000EB0C0008D1
:100030000000000000000000ED0C0008D1090008DD
:10004000EF0C0008F10C0008F30C0008F50C000898
:10005000F70C0008F90C0008FB0C0008FD0C000868
:10006000FF0C0008010D0008030D0008050D000835
:10007000070D0008090D00080B0D00080D0D000804
:100080000F0D0008110D0008130D0008150D0008D4
:10009000170D0008190D00081B0D00081D0D0008A4
:1000A0001F0D0008210D0008230D0008250D000874
:1000B000270D0008290D00082B0D00082D0D000844
:1000C0004543532E46573A30312E30302E303100D2
:1000D0000120C006014908607047C04608ED00E0F5
:1000E00010B51D4CA0688006400F411E032923D87F
:1000F0001A48C0467944097949008F442201171AE9
:10010000E16803220A40032A00D01548E168490645
:10011000490F491C00F031FEE1684904490E48438B
:10012000E168490F491C00F028FE0AE07D2000022A
:1001300007E00120C00304E020688004410F084864
:10014000C84008490860A26892093C231340064A47
:10015000D258D040086010BD0010024000127A0052
:0C0160000024F400000000206C010008E6
:10016C000000000000000000000000000000000083
:10017C000000000000000000000000000000000073
:10018C000100000002000000030000000400000059
:10019C000600000007000000080000000900000035
:1001AC00D0B502AFFFB089B06E4600F037FA01202F
:1001BC000104B160F061C0077060E748006830610D
:1001CC00E64800F02DFB7F280FD080B2E44988422E
:1001DC0003D0E449884200D105E2FC48006831694B
:1001EC00401ADE498842EBD9FDE100F0A4FDDB4862
:1001FC0000F016FB0546401CF9D0A8B2D94988423C
:10020C00DED0FA4800F00CFB0028F0D4FF2319468E
:10021C008143E8B2022813D1022911D1EC4880198C
:10022C00F1694170792101700171F14A1178C17045
:10023C0051780F220A408270052100F083FBD6E72B
:10024C0002460A4321D1F448801979218173922204
:10025C004273822202737322C2726322827243221D
:10026C004272312202722122C27111228271022346
:10027C004371F36903710023C37082700B224270C7
:10028C0001700F2100F05EFBB1E7112813D1112989
:10029C0011D11D4600F04FFD0024DB4804710460B1
:1002AC00052C17D0D14800F0BBFA00289FD4D649B2
:1002BC000855641CF4E701282BD1012929D1D64813
:1002CC008019792101710022C27082701122427052
:1002DC000170B1E7CC4CE078A17862782378534078
:1002EC004B404340206800BA20602079834200D004
:1002FC00C8E000F020FD0024022C46D0BB4800F0E2
:10030C008FFA002800D572E7C34989190855641C77
:10031C00F2E7432823D1432921D100F00CFDB34847
:10032C0000F07EFA002800D561E702460932072169
:10033C008A436946F16069468A1A95467061851C44
:10034C001446B261002D4AD0A84800F069FA002882
:10035C0000D5A3E02070641C6D1EB269F2E7312851
:10036C0032D1312930D100F0E6FC0024A6480471CA
:10037C000460052C70D09D4800F052FA002800D57E
:10038C0035E7A1490855641CF3E7A3488019447864
:10039C006C400078A04275D125460835072085436E
:1003AC0000F0C9FC6846B0616846451BAD46641C4C
:1003BC00EC222846214600F0F7FC2846214600F0A6
:1003CC00C1FAB069854612E700F0BFFC8D480068A1
:1003DC003169401A8549884200D808E703E1716900
:1003EC00481CC9B20346834D002B04D014786140DD
:1003FC00521C5B1EF8E7B269105C814245D1E8687B
:10040C00002803D57C4828607D4828600020B4680B
:10041C00716988423CDC115C06291BD3AA68224214
:10042C00FCD1AA68AA603F22D200EB689343EB6030
:10043C00C900EA680A43EA60EA6802210A43EA60F2
:10044C00EA682243EA60AA682242FCD1EA688A433D
:10045C00EA60B269401CDBE76B4A10785178414086
:10046C0090784840D1784140107981420AD100F00F
:10047C0062FC5E4800F0D4F9002800D5B7E6411CB8
:10048C008A070ED000F061FCB1E600F05EFC05E0DE
:10049C00E86871680843E86000F04DFCF068854638
:1004AC00A5E67061B161F06901025B488019FF2219
:1004BC00F16000F079FC0025504CB069A84209D0DD
:1004CC004A4800F0ADF9002804D45349891948551D
:1004DC006D1CF2E72068C00701D0142000E0042056
:1004EC00F16921507469A54200DC80E63F4800F0B8
:1004FC0097F9002800D57AE600212246A14205DCB6
:10050C00454B9B195B5C5A40491CF7E7D1B28142C1
:10051C00B8D13D49086800BA08603C49884200D20D
:10052C0063E600193A49884200D95EE6F01D19309D
:10053C00F16800F038FC00242E4D7069844213DC05
:10054C00354880190019F11D19310A19314900F08B
:10055C0041FA1034F1E7C046100000208813000067
:10056C00FFFF0000FEFF0000E868002803D52248CA
:10057C00286023482860B069C010F0600021B4687E
:10058C00F068814226DAAA682242FCD1AA68AA60E5
:10059C00B161CA00F31D19339C18606870619B58D7
:1005AC00194805681348C068F4692043B4681149B8
:1005BC00C860AB50A8180D46BFF36F8F71694160CE
:1005CC00A8682042FCD1B169491CD9E71000002071
:1005DC0020010000E868F1698843E860E868716808
:1005EC000843E86001E600F061F9E6E588130000D5
:1005FC0000580140082002402301674514040050B4
:10060C00AB89EFCD10000020040000200030000862
:0C061C00FFEF0108CC0E000820010000D8
:10062800F0B583B06F4800687D21C90000F0A1FBD8
:10063800401E010E0DD16C496C4A50606C4803682D
:100648000B4003218907591801600020906007209A
:100658001060684D2E680020C04301906649674AC3
:100668006F4F0C46BF34106820420AD12868801B9F
:10067800B842F6D33220019900F076F95F4A5E4914
:10068800EFE7506B0327384350635D4A1068B8435F
:10069800106010680C2100918843106010680123D5
:1006A80018431060106804210143116002931D046F
:1006B80054488169C9B2AA2903D08169C9B2CC2931
:1006C80029D1C168002903D54F4901604F4901600C
:1006D800C168490003D54E4941604E49416081696E
:1006E800FF22914381618169EC220A43826181681A
:1006F8002942FCD102994904C2680A43C260816850
:100708002942FCD10299C906C2680A43C260642022
:10071800019900F029F9CF208104052630070268E5
:100728008A4302604521C90402680A430260390508
:10073800C2688A43C260029F3905C2680A43C26020
:100748000F210A02436A934343623A02436A1343FE
:100758004362426AF0239A434262426A1023134377
:1007680043620904426A8A434262416A29434162F8
:10077800B903224A106C0843106427480268BA4338
:1007880002603A070368934303603A03036813431C
:100798000360FA030368934303600268224302601C
:1007A8000268009B1A43026002681C4B13430360F3
:1007B80082680A4382601049C16001683943016058
:1007C8000F4F002E0BD00298B8619624204600F0F7
:1007D800EDF8BD61204600F0E9F8761EF1E703B0B8
:1007E800F0BDC04600000020FFFFFF0010E000E061
:1007F80020ED00E01000002041030000001002403E
:10080800000400500820024023016745AB89EFCD62
:100818003B2A19087F6E5D4C003801400000FF0339
:040828008913000030
:10082C00F0B51E4A146813681D491F4D0E68B606B4
:10083C0011D41668F61A86420DD21668361B4B2E4A
:10084C00F4D314682E68F60701D0142600E00426B1
:10085C0001277751EAE71268D21A82420FD2114867
:10086C000A6812070FD40A6852070ED40A68920756
:10087C000DD40A68D2070CD18868C0B20BE00020F6
:10088C00C043401E07E0082204E0042202E00222DA
:10089C0000E001224A6000B2F0BDC046100000200A
:0C08AC001C380140FFFF00001404005045
:1008B800F0B581B0012002031A490B6813430B609D
:1008C800194B9C6804439C6000241848184D1D4E21
:1008D800AC4205D227583FBA1F602418A419F7E77D
:1008E800144C24681B68A34215D10B6893430B6012
:1008F800124900248C604C600C6072B61049086084
:10090800016881F3088862B640688047E1437D202A
:1009180000F02AF8FAE7FA20074900F025F801B0B4
:10092800F0BDC046381002400030024000300008D8
:10093800FCBF0100FCEF01088813000010E000E094
:0809480008ED00E004D0FFF708
:1009500010B50022054B8A4206DA1C682406FCD535
:10096000845CDC60521CF6E710BDC0461C380140B8
:10097000F0B581B000910546012630040B4F386078
:100980000B4804680A480068001B009988420AD294
:1009900002203860284600F00DF8700438602846C0
:1009A00000F008F8EEE701B0F0BDC04618040050B2
:0409B0001000002013
:1009B40081B005490A6800920A68009BD21A8242F3
:0C09C400FAD301B07047C04610000020BC
:1009D00002480168491C01607047C04610000020B1
:1009E000F0B591B00023102B03D0C45CD4545B1C31
:1009F000F9E7A3480160A34802600022A248102A38
:100A00000BD08B5C835483188C1865785D70A57847
:100A10009D70E478DC70121DF1E704219A4C2C29BA
:100A200048D08D000C22102A06D0A35C10AEB61858
:100A30000C3E3370521CF6E710AEF778B37872783C
:100A40003678880703D00F970E93134612E08F482D
:100A50000D910146865D10A80F96C670CE5D0E966C
:100A60008670CB5C43708A5C0D998E08884FBE5DA2
:100A700056400670844F7A1910461038007870403E
:100A800078550120284316460F3E36785E403E5486
:100A90000220284313460E3B1B780E9E73403B54A6
:100AA000032028430D3A12780F9B5A403A54241DD4
:100AB000491CB4E70A2000F0EFF80920754C0090BB
:100AC00070480068417B427A4273427943784371AF
:100AD000427241708178827A827081728179827BE0
:100AE00082718173C178C279C270C27AC271C27BCD
:100AF000C173C272002104290AD00022102A04D036
:100B0000835CE35C8354121DF8E7401C491CF2E748
:100B10000099080600D1AEE0C8B200F0BDF859480F
:100B2000006807900020102800D1A1E007990A561C
:100B30000F46D109144604921B2211400B460F9018
:100B40006000434059001E4605934BB2DB09134039
:100B500040B2C00910404840410005460690594047
:100B60000E910F98391801200F560B460220095696
:100B70001C4603930846784070400323E3560C93C9
:100B80005840FB0913407C000D9463400A93584081
:100B90006840CB0913404D006B400B935C000194FF
:100BA0006DB2EE0916406640704002960E9B5840AA
:100BB0000A9B5C0065B2EB0913400D9D6DB2ED0917
:100BC0001540654009956C005C4008946040019BAD
:100BD0005BB2DB09134074005C400D9460400C9BD9
:100BE000DC0914405B005C4065006EB2F6091640FB
:100BF0005BB2DB0913406B405A00724050400F9DBE
:100C0000079E70550846049D68400C9E70400A9EE1
:100C100070400B9E7040099E70400E9E7040584080
:100C2000089E70400D9E70405040039E70700F985B
:100C30006F406740174C0E9D6F407940059D69409D
:100C4000099D69405940089D69400D9B594051409C
:100C5000F1700C994F400B994F4006994F40029903
:100C60004F406F400D994F405740B770001D5AE7F5
:100C70000098401E23E7002000F00EF811B0F0BDF0
:100C8000140000200C00002018000020DC0E0008DA
:080C9000C60D0008DC0F00088E
:100C980030B500010A4908180A4909680022042ADF
:100CA8000CD00023042B05D0C45CCD5C6540CD542A
:100CB8005B1CF7E7091D001D521CF0E730BDC0465C
:080CC800180000200C000020C0
:100CD000034C206804348047FBE7FFF767FAFEE720
:040CE000DC1000081C
:060CE400FFF7F4F9F2E74E
:020CEA00FEE723
:020CEC00FEE721
:020CEE00FEE71F
:020CF000FEE71D
:020CF200FEE71B
:020CF400FEE719
:020CF600FEE717
:020CF800FEE715
:020CFA00FEE713
:020CFC00FEE711
:020CFE00FEE70F
:020D0000FEE70C
:020D0200FEE70A
:020D0400FEE708
:020D0600FEE706
:020D0800FEE704
:020D0A00FEE702
:020D0C00FEE700
:020D0E00FEE7FE
:020D1000FEE7FC
:020D1200FEE7FA
:020D1400FEE7F8
:020D1600FEE7F6
:020D1800FEE7F4
:020D1A00FEE7F2
:020D1C00FEE7F0
:020D1E00FEE7EE
:020D2000FEE7EC
:020D2200FEE7EA
:020D2400FEE7E8
:020D2600FEE7E6
:020D2800FEE7E4
:020D2A00FEE7E2
:020D2C00FEE7E0
:0E0D2E0080B50020C143FA20FFF71BFE80BDF8
:060D3C00002000217047B9
:100D420000B581B06846792101700121FFF7FFFDEE
:040D520001B000BD2F
:100D560000B581B068461F2101700121FFF7F5FD3E
:040D660001B000BD1B
:100D6A0080B57D2080000021C943FFF7FCFD80BDCE
:100D7A000A0015D00300400800E052008242FCD964
:100D8A00002000E052089B1A06D340418A42F9D15A
:100D9A00704752089B18F8D200188A42F9D1704756
:080DAA0010B5FFF7C6FF10BDF4
:100DB20000220B0011001A00002A02D0013A8154CD
:040DC200FCD17047A9
:100DC6008D01020408102040801B366CD8AB4D9A6A
:100DD6002F5EBC63C697356AD4B37DFAEFC59139E9
:100DE60072E4D3BD61C29F254A943366CC831D3A13
:100DF60074E8CB8D01020408102040801B366CD8A5
:100E0600AB4D9A2F5EBC63C697356AD4B37DFAEFB5
:100E1600C5913972E4D3BD61C29F254A943366CC2D
:100E2600831D3A74E8CB8D01020408102040801B14
:100E3600366CD8AB4D9A2F5EBC63C697356AD4B371
:100E46007DFAEFC5913972E4D3BD61C29F254A94FC
:100E56003366CC831D3A74E8CB8D0102040810205A
:100E660040801B366CD8AB4D9A2F5EBC63C6973557
:100E76006AD4B37DFAEFC5913972E4D3BD61C29FDE
:100E8600254A943366CC831D3A74E8CB8D0102045F
:100E960008102040801B366CD8AB4D9A2F5EBC6381
:100EA600C697356AD4B37DFAEFC5913972E4D3BDDE
:0F0EB60061C29F254A943366CC831D3A74E8CB02
:040EC800E10000083D
:100ECC00046062063E0B5C4E040620504F34414BCE
:100EDC00637C777BF26B6FC53001672BFED7AB76EB
:100EEC00CA82C97DFA5947F0ADD4A2AF9CA472C096
:100EFC00B7FD9326363FF7CC34A5E5F171D8311503
:100F0C0004C723C31896059A071280E2EB27B27523
:100F1C0009832C1A1B6E5AA0523BD6B329E32F849B
:100F2C0053D100ED20FCB15B6ACBBE394A4C58CF93
:100F3C00D0EFAAFB434D338545F9027F503C9FA867
:100F4C0051A3408F929D38F5BCB6DA2110FFF3D235
:100F5C00CD0C13EC5F974417C4A77E3D645D1973E9
:100F6C0060814FDC222A908846EEB814DE5E0BDBE3
:100F7C00E0323A0A4906245CC2D3AC629195E4791A
:100F8C00E7C8376D8DD54EA96C56F4EA657AAE0874
:100F9C00BA78252E1CA6B4C6E8DD741F4BBD8B8A0F
:100FAC00703EB5664803F60E613557B986C11D9E75
:100FBC00E1F8981169D98E949B1E87E9CE5528DFEC
:100FCC008CA1890DBFE6426841992D0FB054BB1618
:100FDC0052096AD53036A538BF40A39E81F3D7FBA2
:100FEC007CE339829B2FFF87348E4344C4DEE9CBEC
:100FFC00547B9432A6C2233DEE4C950B42FAC34E61
:10100C00082EA16628D924B2765BA2496D8BD12516
:10101C0072F8F66486689816D4A45CCC5D65B692BA
:10102C006C704850FDEDB9DA5E154657A78D9D845E
:10103C0090D8AB008CBCD30AF7E45805B8B345067E
:10104C00D02C1E8FCA3F0F02C1AFBD0301138A6B98
:10105C003A9111414F67DCEA97F2CFCEF0B4E673C8
:10106C0096AC7422E7AD3585E2F937E81C75DF6E76
:10107C0047F11A711D29C5896FB7620EAA18BE1BDC
:10108C00FC563E4BC6D279209ADBC0FE78CD5AF482
:10109C001FDDA8338807C731B11210592780EC5FC8
:1010AC0060517FA919B54A0D2DE57A9F93C99CEF24
:1010BC00A0E03B4DAE2AF5B0C8EBBB3C8353996125
:1010CC00172B047EBA77D626E169146355210C7D63
:1010DC000D11000804000020050000000D1100088F
:1010EC000C000020BC0000001F11000800000020B4
:0C10FC000811000804000000DB0C0008D4
:041108000024F400CB
:10110C00206861680834002200E042540139FCD5A3
:02111C0070471A
:10111E0020686168A2680C3401E08B5C8354013A4C
:04112E00FBD5704736
:0400000508000CE5FE
:00000001FF
